HI-TECH Software C Compiler 

Linker command line:

--edf=C:\Program Files (x86)\HI-TECH Software\PICC\9.83\dat\en_msgs.txt -cs \
  -h+Zadatak 5.sym -z -Q16F690 -ol.obj -MZadatak 5.map -E1 \
  -ACONST=00h-0FFhx16 -ACODE=00h-07FFhx2 -ASTRCODE=00h-0FFFh \
  -AENTRY=00h-0FFhx16 -ASTRING=00h-0FFhx16 -ABANK0=020h-06Fh \
  -ABANK1=0A0h-0EFh -ABANK2=0120h-016Fh \
  -ARAM=020h-06Fh,0A0h-0EFh,0120h-016Fh \
  -AABS1=020h-07Fh,0A0h-0EFh,0120h-016Fh -ACOMMON=070h-07Fh -ASFR0=00h-01Fh \
  -ASFR1=080h-09Fh -ASFR2=0100h-011Fh -ASFR3=0180h-01EFh \
  -preset_vec=00h,intentry,init,end_init -ppowerup=CODE -pfunctab=CODE \
  -ACONFIG=02007h-02007h -pconfig=CONFIG -DCONFIG=2 -AIDLOC=02000h-02003h \
  -pidloc=IDLOC -DIDLOC=2 -AEEDATA=00h-0FFh/02100h -peeprom_data=EEDATA \
  -DEEDATA=2 -DCODE=2 -DSTRCODE=2 -DSTRING=2 -DCONST=2 -DENTRY=2 -k \
  startup.obj Zadatak 5.obj 

Object code version is 3.10

Machine type is 16F690



                Name                               Link     Load   Length Selector   Space Scale
startup.obj     end_init                              0        0        2        0       0
Zadatak 5.obj   config                             2007     2007        1     400E       0
                text714                             982      982       14     1304       0
                text713                             94C      94C       12     1298       0
                text712                             92E      92E        E     125C       0
                text711                             D4F      D4F       7B     1A9E       0
                text710                              1B       1B       A4       36       0
                text709                             CD9      CD9       76     19B2       0
                text708                             922      922        C     1244       0
                text707                             C6D      C6D       6C     18DA       0
                text706                             C07      C07       66     180E       0
                text705                             996      996       14     132C       0
                text704                             93C      93C       10     1278       0
                text703                               4        4       17        8       0
                text702                             95E      95E       12     12BC       0
                text701                             A9D      A9D       33     153A       0
                text700                             A01      A01       25     1402       0
                text699                             A72      A72       2B     14E4       0
                text698                              BF       BF      142      17E       0
                text697                             E50      E50       C6     1CA0       0
                text696                             F16      F16       EA     1E2C       0
                text695                             A26      A26       26     144C       0
                text694                             B0E      B0E       4E     161C       0
                text693                             9E1      9E1       20     13C2       0
                text692                             B5C      B5C       4E     16B8       0
                text691                             DCA      DCA       86     1B94       0
                text690                             201      201      153      402       0
                text689                             9C4      9C4       1D     1388       0
                text688                             917      917        B     122E       0
                text687                             970      970       12     12E0       0
                text686                             A4C      A4C       26     1498       0
                text685                             9AA      9AA       1A     1354       0
                text684                             AD0      AD0       3E     15A0       0
                text683                             BAA      BAA       5D     1754       0
                maintext                            354      354      4AC      6A8       0
                cstackBANK0                          20       20       47       20       1
                cstackCOMMON                         70       70        E       70       1
                cinit                               914      914        3     1228       0
                strings                             800      800       E5     1000       0

TOTAL           Name                               Link     Load   Length     Space
        CLASS   CONST          

        CLASS   CODE           
                end_init                              0        0        2         0
                text714                             982      982       14         0
                text713                             94C      94C       12         0
                text712                             92E      92E        E         0
                text711                             D4F      D4F       7B         0
                text710                              1B       1B       A4         0
                text709                             CD9      CD9       76         0
                text708                             922      922        C         0
                text707                             C6D      C6D       6C         0
                text706                             C07      C07       66         0
                text705                             996      996       14         0
                text704                             93C      93C       10         0
                text703                               4        4       17         0
                text702                             95E      95E       12         0
                text701                             A9D      A9D       33         0
                text700                             A01      A01       25         0
                text699                             A72      A72       2B         0
                text698                              BF       BF      142         0
                text697                             E50      E50       C6         0
                text696                             F16      F16       EA         0
                text695                             A26      A26       26         0
                text694                             B0E      B0E       4E         0
                text693                             9E1      9E1       20         0
                text692                             B5C      B5C       4E         0
                text691                             DCA      DCA       86         0
                text690                             201      201      153         0
                text689                             9C4      9C4       1D         0
                text688                             917      917        B         0
                text687                             970      970       12         0
                text686                             A4C      A4C       26         0
                text685                             9AA      9AA       1A         0
                text684                             AD0      AD0       3E         0
                text683                             BAA      BAA       5D         0
                maintext                            354      354      4AC         0
                cinit                               914      914        3         0

        CLASS   STRCODE        

        CLASS   ENTRY          

        CLASS   STRING         
                strings                             800      800       E5         0

        CLASS   BANK0          
                cstackBANK0                          20       20       47         1

        CLASS   BANK1          

        CLASS   BANK2          

        CLASS   RAM            

        CLASS   ABS1           
                abs_s1                               7E       7E        2         1

        CLASS   COMMON         
                cstackCOMMON                         70       70        E         1

        CLASS   SFR0           

        CLASS   SFR1           

        CLASS   SFR2           

        CLASS   SFR3           

        CLASS   CONFIG         
                config                             2007     2007        1         0

        CLASS   IDLOC          

        CLASS   EEDATA         

        CLASS   BANK3          



SEGMENTS        Name                           Load    Length   Top    Selector   Space  Class     Delta

                reset_vec                      000000  000002  000002         0       0  CODE        2
                text703                        000004  000017  00001B         8       0  CODE        2
                cstackBANK0                    000020  000047  000067        20       1  BANK0       1
                text710                        00001B  0000A4  0000BF        36       0  CODE        2
                cstackCOMMON                   000070  00000E  00007E        70       1  COMMON      1
                text698                        0000BF  000142  000201       17E       0  CODE        2
                text690                        000201  000153  000354       402       0  CODE        2
                maintext                       000354  0004AC  000800       6A8       0  CODE        2
                strings                        000800  0000E5  0008E5      1000       0  STRING      2
                cinit                          000914  000003  000917      1228       0  CODE        2
                text688                        000917  00000B  000922      122E       0  CODE        2
                text708                        000922  00000C  00092E      1244       0  CODE        2
                text712                        00092E  00000E  00093C      125C       0  CODE        2
                text704                        00093C  000010  00094C      1278       0  CODE        2
                text713                        00094C  000012  00095E      1298       0  CODE        2
                text702                        00095E  000012  000970      12BC       0  CODE        2
                text687                        000970  000012  000982      12E0       0  CODE        2
                text714                        000982  000014  000996      1304       0  CODE        2
                text705                        000996  000014  0009AA      132C       0  CODE        2
                text685                        0009AA  00001A  0009C4      1354       0  CODE        2
                text689                        0009C4  00001D  0009E1      1388       0  CODE        2
                text693                        0009E1  000020  000A01      13C2       0  CODE        2
                text700                        000A01  000025  000A26      1402       0  CODE        2
                text695                        000A26  000026  000A4C      144C       0  CODE        2
                text686                        000A4C  000026  000A72      1498       0  CODE        2
                text699                        000A72  00002B  000A9D      14E4       0  CODE        2
                text701                        000A9D  000033  000AD0      153A       0  CODE        2
                text684                        000AD0  00003E  000B0E      15A0       0  CODE        2
                text694                        000B0E  00004E  000B5C      161C       0  CODE        2
                text692                        000B5C  00004E  000BAA      16B8       0  CODE        2
                text683                        000BAA  00005D  000C07      1754       0  CODE        2
                text706                        000C07  000066  000C6D      180E       0  CODE        2
                text707                        000C6D  00006C  000CD9      18DA       0  CODE        2
                text709                        000CD9  000076  000D4F      19B2       0  CODE        2
                text711                        000D4F  00007B  000DCA      1A9E       0  CODE        2
                text691                        000DCA  000086  000E50      1B94       0  CODE        2
                text697                        000E50  0000C6  000F16      1CA0       0  CODE        2
                text696                        000F16  0000EA  001000      1E2C       0  CODE        2
                config                         002007  000001  002008      400E       0  CONFIG      2


UNUSED ADDRESS RANGES

        Name                Unused          Largest block    Delta
        BANK0            0067-006F              9           1
        BANK1            00A0-00EF             50           1
        BANK2            0120-016F             50           1
        CODE             0002-0003              2           2
                         08E5-0913             2F
        CONST            0002-0003              2           2
                         08E5-0913             1B
        EEDATA           2100-21FF            100           2
        ENTRY            0002-0003              2           2
                         08E5-0913             1B
        IDLOC            2000-2003              4           2
        RAM              0067-006F              9           1
                         00A0-00EF             50
                         0120-016F             50
        SFR0             0000-001F             20           1
        SFR1             0080-009F             20           1
        SFR2             0100-011F             20           1
        SFR3             0180-01EF             70           1
        STRCODE          0002-0003              2           2
                         08E5-0913             2F
        STRING           0002-0003              2           2
                         08E5-0913             1B

                                  Symbol Table

??___awdiv                 cstackCOMMON 007B
??___awmod                 cstackCOMMON 0074
??___awtoft                cstackCOMMON 007B
??___ftadd                 cstackBANK0  0020
??___ftdiv                 cstackBANK0  002D
??___ftge                  cstackCOMMON 0076
??___ftmul                 cstackBANK0  0020
??___ftneg                 cstackCOMMON 0073
??___ftpack                cstackCOMMON 0075
??___ftsub                 cstackCOMMON 007E
??___fttol                 cstackCOMMON 0074
??_abs                     cstackCOMMON 007E
??_dinamo                  cstackCOMMON 007E
??_i2c_get_byte            cstackCOMMON 0078
??_i2c_init                cstackCOMMON 007B
??_i2c_open                cstackCOMMON 0077
??_i2c_put_byte            cstackCOMMON 0074
??_i2c_read_ack            cstackCOMMON 0071
??_i2c_read_byte           cstackCOMMON 0071
??_i2c_restart             cstackCOMMON 0070
??_i2c_send_ack            cstackCOMMON 0070
??_i2c_send_address        cstackCOMMON 0075
??_i2c_send_byte           cstackCOMMON 0071
??_i2c_stop                cstackCOMMON 0070
??_i2c_wait_for_SCL        cstackCOMMON 0070
??_init_PIC                cstackCOMMON 0070
??_main                    cstackBANK0  0048
??_read_i2c                cstackBANK0  0022
??_rezultat                cstackBANK0  003A
??_rs232_init              cstackCOMMON 0070
??_rs232_send_byte         cstackCOMMON 0070
??_rs232_send_text         cstackCOMMON 0071
??_start                   cstackCOMMON 0072
?___awdiv                  cstackCOMMON 0077
?___awmod                  cstackCOMMON 0070
?___awtoft                 cstackCOMMON 0078
?___ftadd                  cstackCOMMON 0078
?___ftdiv                  cstackBANK0  0027
?___ftge                   cstackCOMMON 0070
?___ftmul                  cstackCOMMON 0078
?___ftneg                  cstackCOMMON 0070
?___ftpack                 cstackCOMMON 0070
?___ftsub                  cstackBANK0  0027
?___fttol                  cstackCOMMON 0070
?_abs                      cstackBANK0  0027
?_dinamo                   cstackBANK0  002A
?_i2c_get_byte             cstackCOMMON 0076
?_i2c_init                 cstackCOMMON 0079
?_i2c_open                 cstackCOMMON 0076
?_i2c_put_byte             cstackCOMMON 0070
?_i2c_read_ack             cstackCOMMON 0070
?_i2c_read_byte            cstackCOMMON 0070
?_i2c_restart              cstackCOMMON 0070
?_i2c_send_ack             cstackCOMMON 0070
?_i2c_send_address         cstackCOMMON 0074
?_i2c_send_byte            cstackCOMMON 0070
?_i2c_stop                 cstackCOMMON 0070
?_i2c_wait_for_SCL         cstackCOMMON 0070
?_init_PIC                 cstackCOMMON 0070
?_main                     cstackCOMMON 0070
?_read_i2c                 cstackBANK0  0020
?_rezultat                 cstackBANK0  0037
?_rs232_init               cstackCOMMON 0070
?_rs232_send_byte          cstackCOMMON 0070
?_rs232_send_text          cstackCOMMON 0070
?_start                    cstackCOMMON 0070
_ANSEL                     (abs)        011E
_ANSELH                    (abs)        011F
_CARRY                     (abs)        0018
_CREN                      (abs)        00C4
_EEADR                     (abs)        010D
_EECON1                    (abs)        018C
_EECON2                    (abs)        018D
_EEDATA                    (abs)        010C
_FERR                      (abs)        00C2
_GIE                       (abs)        005F
_OERR                      (abs)        00C1
_PORTA                     (abs)        0005
_PORTB                     (abs)        0006
_PORTC                     (abs)        0007
_RA3                       (abs)        002B
_RB4                       (abs)        0034
_RB6                       (abs)        0036
_RCIF                      (abs)        0065
_RCREG                     (abs)        001A
_RCSTA                     (abs)        0018
_RD                        (abs)        0C60
_SPBRG                     (abs)        0099
_SSPCON                    (abs)        0014
_TRISA                     (abs)        0085
_TRISB                     (abs)        0086
_TRISB4                    (abs)        0434
_TRISB6                    (abs)        0436
_TRISC                     (abs)        0087
_TRMT                      (abs)        04C1
_TXREG                     (abs)        0019
_TXSTA                     (abs)        0098
_WR                        (abs)        0C61
_WREN                      (abs)        0C62
__Habs1                    abs1         0000
__Hbank0                   bank0        0000
__Hbank1                   bank1        0000
__Hbank2                   bank2        0000
__Hbank3                   bank3        0000
__Hcinit                   cinit        0000
__Hclrtext                 clrtext      0000
__Hcode                    code         0000
__Hcommon                  common       0000
__Hconfig                  config       2008
__HcstackBANK0             cstackBANK0  0000
__HcstackCOMMON            cstackCOMMON 0000
__Heeprom_data             eeprom_data  0000
__Hend_init                end_init     0002
__Hfunctab                 functab      0000
__Hidloc                   idloc        0000
__Hinit                    init         0000
__Hintentry                intentry     0000
__Hmaintext                maintext     0000
__Hpowerup                 powerup      0000
__Hram                     ram          0000
__Hreset_vec               reset_vec    0000
__Hsfr0                    sfr0         0000
__Hsfr1                    sfr1         0000
__Hsfr2                    sfr2         0000
__Hsfr3                    sfr3         0000
__Hstrings                 strings      0000
__Htext                    text         0000
__Labs1                    abs1         0000
__Lbank0                   bank0        0000
__Lbank1                   bank1        0000
__Lbank2                   bank2        0000
__Lbank3                   bank3        0000
__Lcinit                   cinit        0000
__Lclrtext                 clrtext      0000
__Lcode                    code         0000
__Lcommon                  common       0000
__Lconfig                  config       2007
__LcstackBANK0             cstackBANK0  0000
__LcstackCOMMON            cstackCOMMON 0000
__Leeprom_data             eeprom_data  0000
__Lend_init                end_init     0000
__Lfunctab                 functab      0000
__Lidloc                   idloc        0000
__Linit                    init         0000
__Lintentry                intentry     0000
__Lmaintext                maintext     0000
__Lpowerup                 powerup      0000
__Lram                     ram          0000
__Lreset_vec               reset_vec    0000
__Lsfr0                    sfr0         0000
__Lsfr1                    sfr1         0000
__Lsfr2                    sfr2         0000
__Lsfr3                    sfr3         0000
__Lstrings                 strings      0000
__Ltext                    text         0000
__S0                       (abs)        2008
__S1                       (abs)        007E
__S2                       (abs)        0000
___awdiv                   text709      0CD9
___awdiv@counter           cstackBANK0  0020
___awdiv@dividend          cstackCOMMON 0079
___awdiv@divisor           cstackCOMMON 0077
___awdiv@quotient          cstackBANK0  0022
___awdiv@sign              cstackBANK0  0021
___awmod                   text706      0C07
___awmod@counter           cstackCOMMON 0075
___awmod@dividend          cstackCOMMON 0072
___awmod@divisor           cstackCOMMON 0070
___awmod@sign              cstackCOMMON 0076
___awtoft                  text695      0A26
___awtoft@c                cstackCOMMON 0078
___awtoft@sign             cstackCOMMON 007D
___ftadd                   text698      00BF
___ftadd@exp1              cstackBANK0  0026
___ftadd@exp2              cstackBANK0  0025
___ftadd@f1                cstackCOMMON 0078
___ftadd@f2                cstackCOMMON 007B
___ftadd@sign              cstackBANK0  0024
___ftdiv                   text697      0E50
___ftdiv@cntr              cstackBANK0  0031
___ftdiv@exp               cstackBANK0  0035
___ftdiv@f1                cstackBANK0  002A
___ftdiv@f2                cstackBANK0  0027
___ftdiv@f3                cstackBANK0  0032
___ftdiv@sign              cstackBANK0  0036
___ftge                    text707      0C6D
___ftge@ff1                cstackCOMMON 0070
___ftge@ff2                cstackCOMMON 0073
___ftmul                   text696      0F16
___ftmul@cntr              cstackBANK0  0028
___ftmul@exp               cstackBANK0  0024
___ftmul@f1                cstackCOMMON 0078
___ftmul@f2                cstackCOMMON 007B
___ftmul@f3_as_product     cstackBANK0  0025
___ftmul@sign              cstackBANK0  0029
___ftneg                   text708      0922
___ftneg@f1                cstackCOMMON 0070
___ftpack                  text711      0D4F
___ftpack@arg              cstackCOMMON 0070
___ftpack@exp              cstackCOMMON 0073
___ftpack@sign             cstackCOMMON 0074
___ftsub                   text689      09C4
___ftsub@f1                cstackBANK0  002A
___ftsub@f2                cstackBANK0  0027
___fttol                   text710      001B
___fttol@exp1              cstackCOMMON 007D
___fttol@f1                cstackCOMMON 0070
___fttol@lval              cstackCOMMON 0079
___fttol@sign1             cstackCOMMON 0078
__end_of___awdiv           text709      0D4F
__end_of___awmod           text706      0C6D
__end_of___awtoft          text695      0A4C
__end_of___ftadd           text698      0201
__end_of___ftdiv           text697      0F16
__end_of___ftge            text707      0CD9
__end_of___ftmul           text696      1000
__end_of___ftneg           text708      092E
__end_of___ftpack          text711      0DCA
__end_of___ftsub           text689      09E1
__end_of___fttol           text710      00BF
__end_of_abs               text699      0A9D
__end_of_dinamo            text690      0354
__end_of_i2c_get_byte      text686      0A72
__end_of_i2c_init          text684      0B0E
__end_of_i2c_open          text685      09C4
__end_of_i2c_put_byte      text687      0982
__end_of_i2c_read_ack      text693      0A01
__end_of_i2c_read_byte     text692      0BAA
__end_of_i2c_restart       text704      094C
__end_of_i2c_send_ack      text702      0970
__end_of_i2c_send_address  text688      0922
__end_of_i2c_send_byte     text694      0B5C
__end_of_i2c_stop          text705      09AA
__end_of_i2c_wait_for_SCL  text703      001B
__end_of_init_PIC          text714      0996
__end_of_main              maintext     0800
__end_of_read_i2c          text683      0C07
__end_of_rezultat          text691      0E50
__end_of_rs232_init        text713      095E
__end_of_rs232_send_byte   text712      093C
__end_of_rs232_send_text   text700      0A26
__end_of_start             text701      0AD0
__pcstackBANK0             cstackBANK0  0020
__pcstackCOMMON            cstackCOMMON 0070
__pmaintext                maintext     0354
__pstrings                 strings      0800
__ptext682                 text682      0000
__ptext683                 text683      0BAA
__ptext684                 text684      0AD0
__ptext685                 text685      09AA
__ptext686                 text686      0A4C
__ptext687                 text687      0970
__ptext688                 text688      0917
__ptext689                 text689      09C4
__ptext690                 text690      0201
__ptext691                 text691      0DCA
__ptext692                 text692      0B5C
__ptext693                 text693      09E1
__ptext694                 text694      0B0E
__ptext695                 text695      0A26
__ptext696                 text696      0F16
__ptext697                 text697      0E50
__ptext698                 text698      00BF
__ptext699                 text699      0A72
__ptext700                 text700      0A01
__ptext701                 text701      0A9D
__ptext702                 text702      095E
__ptext703                 text703      0004
__ptext704                 text704      093C
__ptext705                 text705      0996
__ptext706                 text706      0C07
__ptext707                 text707      0C6D
__ptext708                 text708      0922
__ptext709                 text709      0CD9
__ptext710                 text710      001B
__ptext711                 text711      0D4F
__ptext712                 text712      092E
__ptext713                 text713      094C
__ptext714                 text714      0982
__ptext715                 text715      0000
__size_of___awdiv          (abs)        0000
__size_of___awmod          (abs)        0000
__size_of___awtoft         (abs)        0000
__size_of___ftadd          (abs)        0000
__size_of___ftdiv          (abs)        0000
__size_of___ftge           (abs)        0000
__size_of___ftmul          (abs)        0000
__size_of___ftneg          (abs)        0000
__size_of___ftpack         (abs)        0000
__size_of___ftsub          (abs)        0000
__size_of___fttol          (abs)        0000
__size_of_abs              (abs)        0000
__size_of_dinamo           (abs)        0000
__size_of_i2c_get_byte     (abs)        0000
__size_of_i2c_init         (abs)        0000
__size_of_i2c_open         (abs)        0000
__size_of_i2c_put_byte     (abs)        0000
__size_of_i2c_read_ack     (abs)        0000
__size_of_i2c_read_byte    (abs)        0000
__size_of_i2c_restart      (abs)        0000
__size_of_i2c_send_ack     (abs)        0000
__size_of_i2c_send_address (abs)        0000
__size_of_i2c_send_byte    (abs)        0000
__size_of_i2c_stop         (abs)        0000
__size_of_i2c_wait_for_SCL (abs)        0000
__size_of_init_PIC         (abs)        0000
__size_of_main             (abs)        0000
__size_of_read_i2c         (abs)        0000
__size_of_rezultat         (abs)        0000
__size_of_rs232_init       (abs)        0000
__size_of_rs232_send_byte  (abs)        0000
__size_of_rs232_send_text  (abs)        0000
__size_of_start            (abs)        0000
_abs                       text699      0A72
_dinamo                    text690      0201
_exit                      init         0000
_i2c_get_byte              text686      0A4C
_i2c_init                  text684      0AD0
_i2c_open                  text685      09AA
_i2c_put_byte              text687      0970
_i2c_read_ack              text693      09E1
_i2c_read_byte             text692      0B5C
_i2c_restart               text704      093C
_i2c_send_ack              text702      095E
_i2c_send_address          text688      0917
_i2c_send_byte             text694      0B0E
_i2c_stop                  text705      0996
_i2c_wait_for_SCL          text703      0004
_init_PIC                  text714      0982
_main                      maintext     0354
_main$5766                 cstackBANK0  004B
_read_i2c                  text683      0BAA
_rezultat                  text691      0DCA
_rs232_init                text713      094C
_rs232_send_byte           text712      092E
_rs232_send_text           text700      0A01
_start                     text701      0A9D
abs@x                      cstackBANK0  0027
btemp                      (abs)        007E
dinamo@d                   cstackBANK0  0033
dinamo@dt                  cstackBANK0  002D
dinamo@j                   cstackBANK0  0035
dinamo@rez                 cstackBANK0  002A
dinamo@s                   cstackBANK0  0031
dinamo@t                   cstackBANK0  002F
dinamo@temp                cstackBANK0  0037
end_of_initialization      cinit        0914
i2c_get_byte@byte          cstackCOMMON 007A
i2c_get_byte@more          cstackCOMMON 007C
i2c_init@ADRESA1           cstackCOMMON 007B
i2c_init@ADRESA2           cstackCOMMON 0079
i2c_init@ADRESA3           cstackCOMMON 007A
i2c_open@address           cstackCOMMON 0078
i2c_open@mode              cstackCOMMON 0076
i2c_put_byte@data          cstackCOMMON 0074
i2c_read_ack@ack           cstackCOMMON 0072
i2c_read_byte@byte         cstackCOMMON 0075
i2c_read_byte@i            cstackCOMMON 0073
i2c_send_ack@status        cstackCOMMON 0070
i2c_send_address@address   cstackCOMMON 0075
i2c_send_address@rw        cstackCOMMON 0074
i2c_send_byte@byte         cstackCOMMON 0072
i2c_send_byte@i            cstackCOMMON 0073
intlevel0                  functab      0000
intlevel1                  functab      0000
intlevel2                  functab      0000
intlevel3                  functab      0000
intlevel4                  functab      0000
intlevel5                  functab      0000
main@faktor                cstackBANK0  0050
main@high                  cstackBANK0  0059
main@i                     cstackBANK0  004E
main@low                   cstackBANK0  005A
main@x                     cstackBANK0  0061
main@x_max                 cstackBANK0  005B
main@x_min                 cstackBANK0  0053
main@y                     cstackBANK0  0064
main@y_max                 cstackBANK0  005E
main@y_min                 cstackBANK0  0056
read_i2c@ADRESA            cstackBANK0  0025
read_i2c@adr_reg           cstackBANK0  0020
read_i2c@data              cstackBANK0  0024
reset_vec                  reset_vec    0000
rezultat@high              cstackBANK0  0044
rezultat@high_int          cstackBANK0  003C
rezultat@low               cstackBANK0  0037
rezultat@low_int           cstackBANK0  003E
rezultat@mask              cstackBANK0  0043
rezultat@minus             cstackBANK0  0040
rezultat@rez               cstackBANK0  0045
rs232_send_byte@x          cstackCOMMON 0070
rs232_send_text@c          cstackCOMMON 0072
rs232_send_text@i          cstackCOMMON 0074
rs232_send_text@string     cstackCOMMON 0073
start                      init         0000
start@i                    cstackCOMMON 0074
start@x                    cstackCOMMON 0070
start_initialization       cinit        0914
wtemp0                     (abs)        007E
